:1000000025006600050C0200300C06000A0C2700D3
:10001000290506050A0C2A000A0C280049052605B0
:100020000A0C2B009C0C81000307210A61002907A0
:100030001C0AE7021C0A29044907210AE802210ACE
:1000400049040A0243072D0AA6062D0A0A0C2700B6
:10005000290506050A0C2A005D0A0A0C8A004307D6
:100060003A0A29063A0A0F0C270029050604140C3F
:100070002A005D0A140C8A004307470A2906470A2A
:100080000A0C2700290506051E0C2A005D0A1E0C15
:100090008A004307540A2906540A280C2700290518
:1000A0000604280C2A005D0A280C8A0043075D0A12
:1000B00029065D0AA6075D0A6A000B024307690A62
:1000C0008606690A0A0C2800490526050A0C2B0039
:1000D000120A0A0C8B004307760A4906760A0F0CAF
:1000E000280049052604140C2B00120A140C8B005E
:1000F0004307830A4906830A0A0C28004905260596
:100100001E0C2B00120A1E0C8B004307900A490696
:10011000900A280C280049052604280C2B00120AF6
:10012000280C8B004307990A4906990A8607990A01
:040130006B00120A44
:021FFE001A00C7
:00000001FF
